:100000008CC0B1C0B0C0AFC0AEC0B2C0ACC0ABC09D
:10001000AAC0A9C0A8C0A7C0A6C0A5C0A4C0814549
:1000200086468B479048944997609B619E62A16386
:10003000A464A765AA66AC67AE68B069B280B481F3
:10004000B682B883BA84BB84BD84FF21000000005F
:100050000000000000000000000023456C98C9FF6C
:10006000040714233764A0FFFFFFFFFFFFFFFFFF1C
:10007000FFFFFF00000000000000000023405F7A47
:10008000B4FFFFFFFFFFFF001400081400080E1468
:100090000004080E14000305080E140004080A0EDC
:1000A0001114000305080A0E1014000305080A0EB7
:1000B0001012140008000E00080E0004080E0003C1
:1000C00005080E0004080E1100080E1100F3F404D8
:1000D000080E10121400080A0C0E0F10121400085B
:1000E0000EED14000203040500041400040E1400B5
:1000F000040810140004080F1114000305080A0E68
:100100000004080A0E00EEEDECEB140E08040004E7
:10011000080E00EBECEDEEF3F41411241FBECFE556
:10012000D1E0DEBFCDBF20E0A0E6B0E001C01D926F
:10013000A738B207E1F7E2E6F0E085E5808781E0E5
:1001400083831482128287E086831182118688E578
:100150008287612CEDE6F0E08DEF87838EEF85835B
:10016000712CB6D0B5C24CCF1BBC19BC18BC0895BD
:10017000189525B7277E25BF29B7226029BF21E022
:1001800022BF019728F020E188952150E9F7F9CFA7
:10019000089588EE93E0EDCF369A3699FECF95B16B
:1001A0008091600089270895CF93C72D81E0870D46
:1001B0008F73782E662D90E07DD26FEF8C2F90E0BC
:1001C000CF9178C2FF920F931F93CF93DF93F82EB6
:1001D0000CE610E0C5E7D0E0F11005C0CE0162D218
:1001E000F801808304C0F8016081CE0163D22196BA
:1001F00001501109CF37D10579F7DF91CF911F91C8
:100200000F91FF900895D0DF81E0DCCF811101C014
:10021000ABCF815090E0FC01E45BFF4FE491EBBD7C
:10022000FC01E05AFF4FE491E9BDFC01EC58FF4F9F
:10023000849188BD08950F931F93CF93C82F8B018E
:10024000CC2359F085E0E2DFC80193DF8DDFC801E0
:1002500090DFC8018EDFC150F3CFCF911F910F9176
:100260000895EF92FF920F931F93CF93C8E0E82E6B
:10027000F12C062F10E084E1C9DFC7017ADF74DFBB
:10028000C80177DFC150B9F7CF911F910F91FF904F
:10029000EF9008951F93CF93DF938FEA87B986EC91
:1002A00086B91092600010E1C0E0D0E085E090E0F7
:1002B00060DF72DFC80FD11D1150C1F7CE0124E0FD
:1002C000969587952A95E1F7DF91CF911F91089533
:1002D00083EA87B986EC86B93699FECF369A369985
:1002E000FECF85B18095882E8FEF8DBD80E68CBDC9
:1002F0008FE384BB8BE187BB88EE88BB81E083BF43
:1003000091EA9ABD80BF85B7806285BF789487E700
:1003100090E0C8D1853511F076DF11C0712C872DA2
:1003200090E0C0D1682E8F3F19F080E04BDF07C00E
:10033000872D91E0970D792E803488F3F6CF809148
:100340006B001091650000916600D0916300DD2381
:1003500019F000E010E08AE18F5F90E040E050E0AB
:1003600068E870E0882379F09B012F5F3F4FF90127
:100370003197E491EE2319F0922F961BF6CF81501E
:10038000AB01B901EFCF892F612F70E0A92FB0E049
:10039000E82FF0E0002321F09D012E1B3F0B05C04C
:1003A0009F0121503109260F371F3197E40FF51FA8
:1003B000F4902A583F4FF901F082815049F7910F8C
:1003C00090936100112371F0002329F0292F30E070
:1003D0002150310902C020E030E0F901EA58FF4F16
:1003E00081E0808387E0890F282F2150E22FE91BCD
:1003F000F0E0ED5EFE4FE491A22FB0E0AA58BF4FAF
:10040000EC932913F2CFE82FF0E0EB58FF4F21E0F7
:10041000409176003081431320E0821B282F809387
:100420008600862D853F78F5382D313460F48F5F56
:10043000682E891708F0612C809187008F5F8F717B
:100440008093870020C0109287003F3AB0F430912B
:100450006800332311F0DD2331F08F5F682E891798
:1004600090F0612C10C06916E1F3662019F08150FC
:10047000682E09C02150622E06C0D111F2CF8091A2
:100480006400882371F390DE8CE287B986EC86B92C
:100490003699FECF8FEF80936000D62DD53FD0F5F3
:1004A00080918700803138F4E62DF0E0EA58FF4F64
:1004B000C081DC2F2FC06DDE10928700C3E6D0E034
:1004C00000E010E0FF24F39481E0800F0F5F1F4FE6
:1004D00098819F3F29F4219608301105A9F7E4CFB0
:1004E0006DE570E0A8DEF801E359FF4F6080888178
:1004F0008F25888388DE6FE070E080E29CDE888153
:100500008F25888380DE612C44DE80916300882300
:1005100011F3CACF10E000E08CE2E82E96ECD92E61
:10052000CC24CA94DE3E19F463E481E204C0DD3ECB
:1005300021F468E284E195DE75C0DC3E11F469E2E5
:1005400003C0DB3E19F462E581E0F5CFD33F41F40F
:1005500084E15CDE8AE090E00CDE88E057DE3CC09F
:10056000D43F51F584E690E004DE16DE90E0292FBA
:1005700030E0F901E25EFF4FE491E81710F49E5F6E
:10058000F6CFF901E15EFF4FF4906DE770E08F2D3B
:100590008295869587704FDE8EEE92E0EADD65E00B
:1005A00070E081E048DE85E694E0E3DD6DE770E031
:1005B0008F2D8F7140DE0FC0DE3F81F4612CF12C56
:1005C000F0926B0020DE6AEF70E081E034DEF3949D
:1005D000FAE1FF12F5CFDDDDDCDD24C0DD3F79F58A
:1005E000612C8FEF80936C000EDE85E00FDED1DD95
:1005F000D0DD84E10BDE4EDE80936C0004DEC9DDCD
:10060000C8DDF9CF3699FECFC092600020916C0012
:100610002817F8F40F5F0930C0F484EF91E0A9DDEA
:1006200010928700B9DD803908F03AC01F5F18309A
:1006300008F478CFC531C8F010E0CAE0DAE08C2FBA
:10064000E5DD28DEE7B8D6B8DDCFC33030F3C150E2
:100650000AC090E030E022503109821793071CF461
:10066000CD1708F4CF5F00E0D8CFC23030F08C2F28
:1006700086958695C695C80F12C076DD85B7877EAC
:10068000806185BFF89485B7846885BF8B7F85BFFF
:1006900085B7806285BF889585B78F7D85BFDC2F44
:1006A00010E040CFE199FECF1FBA8EBBE09A9927A8
:1006B0008DB30895262FE199FECF1CBA1FBA8EBBC9
:1006C0002DBB0FB6F894E29AE19A0FBE01960895F9
